:020000020000FC
:020000005EC0E0
:02001400A6C381
:02001800AAC27A
:02003C00B1C24F
:02007400CBC2FD
:1000BC0058C1A89501E20EBF0FEF0DBF07E104B9BF
:1000CC0008E605B901E00DBD00E50CBD289A2C9899
:1000DC00179A0F9A0CE000936A0000E20DBB0AEA33
:1000EC00A02E01EBB02EEE27CC27F2E0D2E0B5E04B
:1000FC00AA277FEF30E82227EE249EE10FE30BB90D
:10010C00A89500E004BF0EE10093600006E00093A8
:10011C00600054E0D5D117980000000000000000EA
:10012C00000000000000000000000000179A54E0DE
:10013C00C7D101E000937E0000EC00937C00A198F5
:10014C002F98A09A999A989A279AA09A06E00093C9
:10015C00810000E20093B60006E00093B10000912C
:10016C00B6000F71E1F707E007BB01E000937000E8
:10017C00689A74984ED204D103EC2898AED100271B
:10018C00ACD1289A00EE2898A8D108EBA6D1289AD1
:10019C0001EE2898A2D10AEAA0D1289A02EE28985A
:1001AC009CD10DEC9AD1289A03EE289896D10BEAA3
:1001BC0094D1289A08EC289890D106E38ED1289AED
:1001CC0005EC28988AD100E888D1289A0CEE28985A
:1001DC0084D108E382D1289A0EEE28987ED105E0CE
:1001EC007CD1289A0DEE289878D100EC76D1289AFB
:1001FC000EEC289872D108E070D1289A0FE8289854
:10020C006CD1289A0FEF0CBB7894D8D0FD1334C066
:10021C00EC1332C013B1107680E61827832F80764A
:10022C008117A1F33B793860312BE12A103629F084
:10023C00103461F01032A9F0377918E010932101D5
:10024C0010E0109373002F98A09AE0CF18E0109351
:10025C00210110E010937300A098A19A2F9A31609D
:10026C00D5CF18E01093210110E010937300A098E3
:10027C00A1982F9A3E7FCACF1191112E183069F593
:10028C0011911A94183049F511911A9411911A94EC
:10029C0011911A94183009F020C011911A9433FD61
:1002AC001CC0183001F1163089F11A3029F11C30BC
:1002BC00A1F411911A94123088F11E3FB0F511502F
:1002CC00612E1E5F712E346018E01093210110E036
:1002DC00109373002F98A09A00C010E0E10DF11F4D
:1002EC00F2FDF2E093CF3B7F11911A9426D0A098A7
:1002FC00A19A2F9A3160F1CF18E01093210110E0F0
:10030C00109373003B7F2F98A09AE7CF3A7F1191FF
:10031C001A9413D0A098A1982F9ADFCF3A7F1FEF91
:10032C000CD0A098A1982F9AD8CF3B7F1FEF05D067
:10033C00A098A19A2F9A3160D0CF612F15E010931D
:10034C00290110E01093280110932501109324012A
:10035C001FE21ABB12E0109373001DE010932101F1
:10036C0008950FB70F936A9541F42F98A09A08E05F
:10037C000093210100E0009373000F910FBF1895BB
:10038C0002EC2898AAD008E0A8D0289A01E828986E
:10039C00A4D000E0A2D0289A0830C1F7089502EC4E
:1003AC0028989BD009E099D0289A01E8289895D0F4
:1003BC0000E093D0289A0930C1F7089502EC2898F0
:1003CC008CD006E18AD0289A01E8289886D000E0E3
:1003DC0084D0289A0631C1F7089502EC28987DD074
:1003EC0009E17BD0289A01E8289877D000E075D0F5
:1003FC00289A0931C1F70895243079F500E06DD0C1
:10040C0000E06BD000E069D000E067D000E065D080
:10041C00B02E00E062D0A02E289A229720E139D08D
:10042C00A2D2089507E8289858D000E056D0D02ED4
:10043C00289A00E2289851D000E04FD0065009933A
:10044C000350002E00E049D000E047D000E045D03A
:10045C000993063089F2083019F0289A22970895EA
:10046C0000E03BD000E039D000E037D000E035D0E0
:10047C0000E033D009930A94D9F700E02ED000E0C5
:10048C002CD000E02AD0289A0993D992D2FDD2E040
:10049C00089501E8289821D000E01FD0289A013156
:1004AC00C1F30F31B1F30231A1F379DF0FE82898D2
:1004BC0014D000E012D0289A03FDB4DF8EDF08952B
:1004CC004FEF11D000000000000000000000000001
:1004DC00000000005A95A1F708950EBD0DB507FF59
:1004EC00FDCF0EB5089500000000000000000000D4
:1004FC000000000000004A95B1F7089502E8289822
:10050C00ECDF00E0EADF289A007E003638F021307C
:10051C00B9F40DD222E00F910FBF189540DF4EDFDA
:10052C00223081F424E0A89504B7077F04BF0EE1C4
:10053C000093600006E0009360000F910FBF1895C8
:10054C002EDF3CDFEE2420E0A89504B7077F04BF24
:10055C000EE10093600006E0009360000F910FBF66
:10056C0018950FB70F930FE82898B7DF289A01E872
:10057C002898B3DF00E0B1DF289A063139F0013159
:10058C0029F00F31A1F3023191F3B8CF4BDF0F916A
:10059C000FBF18950FB70F939A9519F00F910FBFC6
:1005AC001895A8950EE1009360000EE00093600092
:1005BC001F93809084009090850000270093850005
:1005CC000093840032FF04C0961460F0971488F4F2
:1005DC00E32A8AD00FED00937A009EE11F910F91D0
:1005EC000FBF189518E0A9DEA098A19A2F9A316038
:1005FC00EFCF18E0A2DEA098A1982F9A3E7FE8CF0B
:10060C000FB70F9350907800209079000F910FBF87
:10061C00189551D132D1709A0000000070980000EA
:10062C000000709A00000000709800000000709AA2
:10063C0000000000709800000000709A000000009C
:10064C00709800000000709A0000000070986C9880
:10065C00000000000000000000000000709A000084
:10066C000000709800000000709A00000000709864
:10067C006C9A709A00000000709813D16C9A709A62
:10068C0000000000709800000000709A000000004C
:10069C00709800000000709A000000007098000034
:1006AC000000709A00000000709800000000709A22
:1006BC0000000000709800000000709A000000001C
:1006CC00709800000000709A0000000070986C9800
:1006DC00000000000000000000000000709A000004
:1006EC0000007098DED00895C8D0709A0000000009
:1006FC00709800000000709A0000000070980000D4
:10070C000000709A00000000709800000000709AC1
:10071C0000000000709800000000709A00000000BB
:10072C00709800000000709A0000000070986C989F
:10073C00000000000000000000000000709A0000A3
:10074C000000709800000000709A00000000709883
:10075C00A8D0EC9A08950FB70F9366F0EC985DD083
:10076C0055D0302E5AD04DD0402E10D00F910FBFF7
:10077C006894189552D04AD050D043D0C02E21E066
:10078C0088DEF1D00F910FBFE894189576D0709A4F
:10079C0000000000709800000000709A000000003B
:1007AC00709800000000709A000000007098000023
:1007BC000000709A00000000709800000000709A11
:1007CC000000000070986C98000000000000000011
:1007DC0000000000709A0000000070986C9A709AEB
:1007EC000000000070986C980000000000000000F1
:1007FC0000000000709A00000000709852D0EC9A33
:10080C000895709A00000000709808956C9A709A80
:10081C000000000070986C9808950027709A6499F5
:10082C000068709800000000709A649900647098D9
:10083C0000000000709A649900627098000000003B
:10084C00709A64990061709800000000709A649925
:10085C000860709800000000709A649904607098A9
:10086C0000000000709A649902607098000000000B
:10087C00709A64990160709808956C987098000053
:10088C000000709A6C9A709800000000709A6C9836
:10089C0000000000000000000000000070986C9A3E
:1008AC0008956C986499FECF709A000000007098BF
:1008BC00649BFECF08956C98709A000000007098AD
:1008CC0000000000709A000000007098000000000A
:1008DC00709A00000000709800000000709A0000F0
:1008EC000000709800000000709A000000007098E2
:1008FC0000000000709A00000000709800000000DA
:10090C00709A00000000709800000000709A0000BF
:10091C000000709800000000709A000000007098B1
:10092C0000000000709A00000000709808952C9A46
:10093C0000002C9800E62898D0DD0BE0CEDD00E41A
:10094C00CCDD08E8CADD01E0C8DD0DECC6DD0BEA44
:10095C00C4DD0FEFC2DD0FEFC0DD08EBBEDD0AEA30
:10096C00BCDD289A08952C9A00002C9800E6289853
:10097C00B4DD03E1B2DD01E6B0DD08E8AEDD07E091
:10098C00ACDD0DECAADD0BEAA8DD0B2DA6DD0A2DE6
:10099C00A4DD08EBA2DD0AEAA0DD0E2D9EDD0C2DF8
:1009AC009CDD042D9ADD032D98DD082D96DD092D97
:0E09BC0094DD052D92DD022D90DD289A089520
:00000001FF
